:10000000C5C00000DEC00000DCC00000DAC0000097
:10001000D8C00000D6C00000D4C00000D2C000008C
:10002000D0C00000CEC00000D8C10000F7C1000061
:10003000C8C00000C6C00000C4C00000C2C00000AC
:10004000C0C00000BEC00000BCC00000BAC00000BC
:10005000B8C00000B6C00000B4C00000B2C00000CC
:10006000B0C00000AEC00000ACC00000AAC00000DC
:10007000A8C00000A6C00000A4C00000A2C00000EC
:10008000A0C000009EC000009CC000009AC00000FC
:1000900098C0000096C0000094C0000092C000000C
:1000A00090C000008EC000008CC000008080000066
:1000B000010000E6001200020000F800220021000A
:1000C000000A0109002200001A012B00030000456C
:1000D000010401030904490116020309046101280E
:1000E00001C1360000001201100100000040C016DE
:1000F000DC27000101020001090222000101008049
:10010000320904000001030000000921110100016F
:10011000222B000705810340000A05010905A10102
:100120000901A10009300931150026FF0075089565
:10013000028102C005091901290815002501750170
:1001400095088102C00403090416034A006F007376
:1001500000680020004B0072006F00700066000015
:100160000028035400650065006E007300790020CC
:100170000053004E00450053002000470061006D11
:1001800000650070006100640000000011241FBEC3
:10019000CFEFDAE0DEBFCDBF11E0A0E0B1E0E6E8EE
:1001A000F6E002C005900D92A230B107D9F711E038
:1001B000A2E0B1E001C01D92A730B107E1F793D0F2
:1001C00060C21ECF599880E090E04FEF5898589A3F
:1001D00021E04A9920E08630910509F45AC0873021
:1001E0009105BCF48330910509F43FC0843091053A
:1001F0004CF4322F31708130910541F182309105FC
:1002000001F52BC084309105D1F185309105C9F4F9
:100210003BC08930910509F44AC08A3091053CF40D
:1002200087309105D9F18830910559F43CC0322FBF
:1002300031708A30910509F440C08B30910509F482
:1002400042C0220F309106013D7F15C0330F330F9E
:10025000330F20910601277F3CC03295330F330FB7
:10026000307C209106012F7B34C0279522272795CB
:10027000309106013F77322B309306012DC02223A7
:1002800059F11092050128C0222331F14093050154
:1002900023C0222309F1109204011EC02223E1F0A1
:1002A0004093040119C0309106013E7FE4CF220F34
:1002B000220F309106013B7FDECF3295307F2091B7
:1002C00006012F7E06C03295330F307E2091060145
:1002D0002F7D232B2093060101968C30910509F088
:1002E00075CF599A089580E880936100109261005B
:1002F000509A519A589A599A52985A98569A5E9A80
:1003000016D02CD08823E9F380E197E220E931E090
:10031000F9013197F1F70197D9F75E9822D052DFB2
:1003200027D0FCCF8091E80080FFFCCF089581E0CA
:100330008093D70080EA8093D80082E189BD09B418
:1003400000FEFDCF80E98093D8001092E00010926B
:1003500002018CE08093E20078940895809102017C
:10036000089584E091E06CEA70E043E050E080C1E1
:1003700080910201882369F18FB7F89491E09093FE
:10038000E9009091E4009E5C21E03091E80035FFA7
:1003900012C0909104019093F10090910501909307
:1003A000F100909106019093F1009AE39093E80098
:1003B0008FBF80E008958FBF80910201882349F0AC
:1003C0008091E400891739F08FB7F8942093E90001
:1003D000DCCF8FEF08958FEF08951F920F920FB625
:1003E0000F9211248F938091E1001092E10083FF1E
:1003F0000FC01092E90081E08093EB001092EC00B6
:1004000082E38093ED0088E08093F0001092020177
:100410008F910F900FBE0F901F9018951F920F9203
:100420000FB60F921124EF92FF921F932F933F93D9
:100430004F935F936F937F938F939F93AF93BF93EC
:10044000CF93DF93EF93FF931092E9008091E80040
:1004500083FFF5C03091F1002091F1008091F1000F
:10046000C82FD0E04091F100942F80E0C82BD92B09
:100470006091F10070E04091F100942F80E0682BD2
:10048000792BA091F1001091F10082EF8093E800A8
:10049000263009F051C047E02FEA30E0F90185919C
:1004A00094918C179D0739F4F901329685919491B6
:1004B0008617970729F0295F3F4F415079F7BFC052
:1004C000F901349685919491AC012A5F3F4FF9016F
:1004D0002491B0E0912F80E0A82BB92BAF3FB1055C
:1004E00019F010F0AFEFB0E0A21708F42A2FAEEF2A
:1004F0008091E80090E0BC01657070706115710535
:10050000B9F382FD9FC0322F213408F030E4CA01D4
:10051000632F06C0FC010196E491E093F100615065
:100520006623C1F7430F511D231BA093E80022232C
:10053000F9F63034E9F286C0253049F48EEF809325
:10054000E800F0DE9E0120682093E3007BC02930A4
:1005500059F5332309F038C0C09302018EEF809320
:10056000E80041E080EE90E04093E9009C012F5FBD
:100570003F4FFC0154915093EB00552359F0F90182
:1005800024912093EC00FC0132960396E491E093D1
:10059000ED0001C0C9014F5F453031F78EE1809316
:1005A000EA001092EA004EC0283031F4303861F48D
:1005B000B9DE8091020126C0222331F4B3DE10920D
:1005C000F1001092F10037C061157105C1F5313AA3
:1005D000E1F4213061F4A6DE809104018093F10002
:1005E000809105018093F100809106010BC02230BB
:1005F00021F498DE8091030105C0233001F592DEDD
:10060000809100018093F10016C03132C1F429308D
:1006100041F48091E80082FFFCCF8BEF8093E800EB
:100620000AC02A3021F47E01F092030104C02B306D
:1006300031F4C09300018EEF8093E80003C081E2A3
:100640008093EB00FF91EF91DF91CF91BF91AF913C
:100650009F918F917F916F915F914F913F912F91DA
:100660001F91FF90EF900F900FBE0F901F90189565
:10067000FB01DC0102C005900D9241505040D8F7BB
:060680000895F894FFCF7D
:02068600010071
:00000001FF
